:020000040800F2
:10100000EA320E024C554D454E4945523100000022
:101010000000000001010000100008183001640FFA
:10102000001E0000000064000100E803DC05D0079A
:101030006400800C000000000E00000000000000B2
:101040000000646661230000000000000000000052
:101050000000000000000000000000000000000090
:101060000000000000000000000000000000000080
:101070000000000000000000000000000000000070
:101080000000000000000000000000000000000060
:101090000000000000000000000000000000000050
:1010A0000000000000000000000000000000000040
:1010B0000000000000000000000000000000000030
:1010C0000000000000000000000000000000000020
:1010D0000000000000000000000000000000000010
:1010E0000000000000000000000000000000000000
:1010F00000000000000000000000000000000000F0
:1011000000000000000000000000000000000000DF
:1011100000000000000000000000000000000000CF
:1011200000000000000000000000000000000000BF
:1011300000000000000000000000000000000000AF
:0811400000001932000000005C
:1014000000200020B55A0008B35A0008A94300087C
:1014100000000000000000000000000000000000CC
:10142000000000000000000000000000B35A0008A7
:10143000000000000000000049430008314200089D
:10144000B15A0008B15A0008B15A0008B15A000850
:10145000B15A0008B15A0008B15A0008B15A000840
:10146000B15A000885170008ED4E0008F93B000846
:10147000B15A00080D170008411700082140000864
:10148000ED3B0008B15A0008B15A0008B15A0008F3
:10149000B15A0008B15A0008B15A0008B15A000800
:1014A000B15A0008B15A0008B15A0008814E00082C
:1014B000B15A0008B15A0008B15A0008B15A0008E0
:1014C00038B5704C704A4FF0FF33E360236100235E
:1014D000E36023616D4B636144F60123A36140F631
:1014E0001103E3614FF0E023C3F8082D636823F094
:1014F0000203636063681A07FCD4236823F08073D7
:10150000236023689B01FCD4614B6360236843F034
:101510008073236023689D01FCD5636843F0020358
:1015200063604FF090434FF000521A6240F2222263
:101530005A622222C3F820244FF48055554AC3F83A
:101540000C541A60544AC3F80024E26942F00202C3
:10155000E261D3F8202442F48032C3F82024D3F887
:101560000C2442F48072C3F80C24D3F8002422F433
:101570008072C3F800244021102004F0F3FA802187
:101580001B2004F0EFFA40211C2004F0EBFA80212C
:10159000092004F0E7FA80210A2004F0E3FA402150
:1015A0000B2004F0DFFA0D2004F0D0FA0E2004F036
:1015B000CDFA0F2004F0CAFA102004F0C7FA142064
:1015C00004F0C4FA1B2004F0C1FA1C2004F0BEFA97
:1015D000092004F0BBFA0A2004F0B8FA0B2004F04A
:1015E000B5FA2E4B0222C3F80C2C1022C3F8082C9B
:1015F0004FF0804240215160782191614FF4807119
:10160000D1611562626B42F001026263626B900706
:10161000FCD5234AC3F80824224A6721D162092154
:1016200011601168C907FCD4D3F8082442F0040201
:10163000C3F80824D3F808245207FBD44FF480726F
:10164000C3F804244FF0FF32C3F80C241649C3F842
:1016500010240322C3F8342401220A70D3F834245E
:1016600042F48C42C3F834240A780232D2B20A70AF
:10167000013A1205C3F82C240C4B0D4A1A610D4A8D
:101680005A6138BD00100240001400080500060031
:1016900000002408FFBFEAEBFAEFFFFF0020014043
:1016A00001008000001000400C02002000000240F9
:1016B0004C2401400002002000F00303013B022BF8
:1016C0009ABF054AD35600234207044A48BF43F451
:1016D0000063D361704700BFA05B000800000140B9
:1016E000074B9A68D2070AD4064A1278DA6040F2A9
:1016F00083529A60A3F56043034AC3F808247047F5
:10170000000002400C02002001019E000A4BD3F8A9
:10171000102CD1070BD56FF00101C3F8101CD3F8C2
:10172000403C23B10549CB6923F4E063CB619306C8
:1017300001D502F049BC7047002001400000014083
:101740000D4BD3F8101CC80608D50C486FF01002DA
:10175000C3F8102CC26942F48062C26189070AD5BD
:101760006FF00202C3F8102CD3F80824D20544BF4E
:10177000034AC3F8082470470020014000000140DC
:101780000101DE00114A022313B553600023936068
:101790000F4C10491048A2F56042C2F80814A18805
:1017A000B0FBF1F1608822880093484300134A435C
:1017B000C0F5B4604FF4FA614843C01212131946E1
:1017C000643002F08BFC02B010BD00BF000002408C
:1017D000000200200100800050FB4A00044B1A6800
:1017E000002A04DB0028A2BF024A1860106070477C
:1017F000480100208001002070B505460E460024F7
:1018000056F8240018B1294604F020F808B92046FB
:1018100070BD0134F4E713B50A220C4601A904F0A7
:10182000F5F8019B1B781BB92060012002B010BDA8
:101830000020FBE710B50446006803F0FDFF2060C0
:1018400010BD0000F0B585B00A2204460D4664279D
:1018500091FBF7F601A9304603F0C6FF014620468A
:10186000FFF7E8FF0D492046FFF7E4FF07FB16509E
:101870000A2201A903F0B8FF04F017F8084E054644
:10188000012D05DD01A92046FFF7D4FF05B0F0BD0D
:1018900031462046FFF7CEFF0135F1E7745E0008C0
:1018A000765E00081FB504460A22084601A903F027
:1018B0009BFF01462046FFF7BDFF04B010BD0000AE
:1018C000F0B58DB0464F0190054602AE0024394672
:1018D00001A803F0F2FF18B954B920460DB0F0BDCD
:1018E0000378002BF3D001340A2C46F8040BEED118
:1018F0003C4902980195FFF77FFF092801F2B28366
:10190000DFE810F00A0015009800AE036807A70B87
:10191000B30BB80BD10BE60B334901A8FFF78AFFD5
:10192000324901A8FFF786FF019C641BD5E7012C13
:1019300041F098832E4C2F4901A8FFF77BFFA07838
:10194000FFF74CFF014601A8FFF7ACFF2A4901A8A9
:10195000FFF770FFE17801A8FFF7A4FF274901A86E
:10196000FFF768FF211D01A8FFF764FF2449254CFC
:1019700001A8FFF75FFF244B01A81968FFF792FF4A
:1019800023683BB1214901A8FFF754FF216801A852
:10199000FFF788FF1E4901A8FFF74CFF1D4B01A868
:1019A0001968FFF74FFF1C4901A8FFF743FF1B4BC6
:1019B00001A81968FFF746FF194901A8FFF73AFF88
:1019C000184B01A81968FFF76DFF174901A8FFF729
:1019D00031FF164B196801A8FFF764FF14499CE713
:1019E000785E0008EC6000087D5E0008B0600008CA
:1019F00000000020E55E0008745E0008F25E00084A
:101A0000F55E00080C07002008070020FE5E0008B5
:101A1000065F0008280700200F5F0008BC060020B2
:101A2000185F0008B8060020215F0008CC060020DF
:101A30007B5E0008012C41F01583AD4CAD4901A837
:101A4000FFF7F8FEAC4901A8FFF7F4FE217D01A8DD
:101A5000FFF728FFA94901A8FFF7ECFEA84901A854
:101A6000FFF7E8FEA44901A8FFF7E4FE617D01A8A5
:101A7000FFF718FFA14901A8FFF7DCFEA14901A863
:101A8000FFF7D8FE9C4901A8FFF7D4FEA17D01A86D
:101A9000FFF708FF994901A8FFF7CCFE9A4901A872
:101AA000FFF7C8FE944901A8FFF7C4FEE17D01A835
:101AB000FFF7F8FE914901A8FFF7BCFE934901A882
:101AC000FFF7B8FE8C4901A8FFF7B4FE217E01A8FC
:101AD000FFF7E8FE894901A8FFF7ACFE8C4901A891
:101AE000FFF7A8FE844901A8FFF7A4FE617E01A8C4
:101AF000FFF7D8FE814901A8FFF79CFE854901A8A0
:101B0000FFF798FE7C4901A8FFF794FEA17E01A88B
:101B1000FFF7C8FE794901A8FFF78CFE7E4901A8AE
:101B2000FFF788FE744901A8FFF784FEE17E01A853
:101B3000FFF7B8FE714901A8FFF77CFE774901A8BD
:101B4000FFF778FE6C4901A8FFF774FE217F01A81A
:101B5000FFF7A8FE694901A8FFF76CFE704901A8CC
:101B6000FFF768FE644901A8FFF764FE617F01A8E2
:101B7000FFF798FE614901A8FFF75CFE694901A8DB
:101B8000FFF758FE5C4901A8FFF754FEA17F01A8AA
:101B9000FFF788FE594901A8FFF74CFE624901A8EA
:101BA000FFF748FE544901A8FFF744FEE17F01A872
:101BB000FFF778FE514901A8FFF73CFE5B4901A8F9
:101BC000FFF738FE4C4901A8FFF734FE94F82010C7
:101BD00001A8FFF767FE494901A8FFF72BFE54490A
:101BE00001A8FFF727FE444901A8FFF723FE94F858
:101BF000211001A8FFF756FE404901A8FFF71AFE81
:101C00004C4901A8FFF716FE3B4901A8FFF712FE59
:101C100094F8221001A8FFF745FE384901A8FFF704
:101C200009FE454901A8FFF705FE334901A8FFF762
:101C300001FE94F8231001A8FFF734FE2F4901A8F4
:101C4000FFF7F8FD3D4901A8FFF7F4FD2A4901A877
:101C5000FFF7F0FD94F8241001A8FFF723FE2749B1
:101C600001A8FFF7E7FD364901A8FFF7E3FD224988
:101C700001A8FFF7DFFD94F8251001A8FFF712FE79
:101C80001E4901A8FFF7D6FD2E4901A8FFF7D2FD96
:101C9000194901A8FFF7CEFD94F8261001A8FFF717
:101CA00001FE164901A8FFF7C5FD274901A8FFF766
:101CB000C1FD114901A8FFF7BDFD94F8271001A847
:101CC000FFF7F0FD0D4901A8FFF7B4FD1F4901A87A
:101CD000FFF7B0FD084901A8FFF7ACFD94F8281004
:101CE00001A8FFF7DFFD054901A8FFF7A3FD2FE0DD
:101CF000000000202C5F0008295F00087B5E0008C0
:101D0000305F0008355F00083C5F0008445F000852
:101D10004B5F0008565F0008615F00086A5F0008BB
:101D2000735F00087C5F0008855F00088F5F000814
:101D3000995F0008A35F0008AD5F0008B75F000867
:101D4000C25F0008CC5F0008D65F0008E05F0008B3
:101D5000AC4901A8FFF76EFDAB4901A8FFF76AFD8A
:101D6000618D01A8FFF79EFDA84901A8FFF762FD5C
:101D7000A74901A8FFF75EFDA34901A8FFF75AFD97
:101D8000A18D01A8FFF78EFDA04901A8FFF752FD24
:101D9000A04901A8FFF74EFD9B4901A8FFF74AFDA6
:101DA000E18D01A8FFF77EFD984901A8FFF742FDEC
:101DB000994901A8FFF73EFD934901A8FFF73AFDB5
:101DC000218E01A8FFF76EFD904901A8FFF732FDB3
:101DD000924901A8FFF72EFD8B4901A8FFF72AFDC4
:101DE000618E01A8FFF75EFD884901A8FFF722FD7B
:101DF0008B4901A8FFF71EFD834901A8FFF71AFDD3
:101E000094F8341001A8FFF74DFD804901A8FFF7B1
:101E100011FD844901A8FFF70DFD7B4901A8FFF7DB
:101E200009FD94F8351001A8FFF73CFD774901A89A
:101E3000FFF700FD7C4901A8FFF7FCFC724901A8EF
:101E4000FFF7F8FC94F8361001A8FFF72BFD6F4957
:101E500001A8FFF7EFFC754901A8FFF7EBFC6A4901
:101E600001A8FFF7E7FC94F8371001A8FFF71AFD67
:101E7000664901A8FFF7DEFC6D4901A8FFF7DAFC0F
:101E8000614901A8FFF7D6FC94F8381001A8FFF7C4
:101E900009FD5E4901A8FFF7CDFC664901A8FFF7DF
:101EA000C9FC594901A8FFF7C5FC618F01A8FFF7DC
:101EB000F9FC564901A8FFF7BDFC5F4901A8FFF7EF
:101EC000B9FC514901A8FFF7B5FC94F83C1001A8F2
:101ED000FFF7E8FC4D4901A8FFF7ACFC574901A802
:101EE000FFF7A8FC484901A8FFF7A4FC94F83D10AF
:101EF00001A8FFF7D7FC454901A8FFF79BFC504913
:101F000001A8FFF797FC404901A8FFF793FC94F85C
:101F10003E1001A8FFF7C6FC3C4901A8FFF78AFC68
:101F2000484901A8FFF786FC374901A8FFF782FC62
:101F300094F83F1001A8FFF7B5FC344901A8FFF75A
:101F400079FC414901A8FFF775FC2F4901A8FFF76B
:101F500071FCB4F8401001A8FFF7A4FC2B4901A8BC
:101F6000FFF768FC394901A8FFF764FC264901A87E
:101F7000FFF760FC04F1420101A8FFF75BFC234975
:101F800001A8FFF757FC324901A8FFF753FC1E498F
:101F900001A8FFF74FFC94F8421101A8FFF782FC5B
:101FA0001A4901A8FFF746FC2A4901A8FFF742FC9D
:101FB000154901A8FFF73EFC94F8431101A8FFF76B
:101FC00071FC124901A8FFF735FC234901A8FFF76E
:101FD00031FC0D4901A8FFF72DFC94F8441101A82C
:101FE000FFF760FC094901A8FFF724FC1B4901A881
:101FF000FFF720FC044901A8FFF71CFC94F84511E9
:10200000E9E400BFEA5F0008295F00087B5E000882
:10201000F45F0008FE5F0008086000081360000815
:102020001E60000829600008346000083F60000856
:102030004A60000856600008616000086B60000894
:10204000756000087F6000088A60000894600008DE
:102050009A600008A1600008A8600008AC60000851
:10206000022C40F0FF8797490398FFF7C5FB29280A
:1020700000F2F887DFE810F02A003F005200650008
:1020800078008B009E00B100C400D700EA00FD007C
:10209000100148015D01720187019C01B101C60177
:1020A000DB01F0010302160229023C024F02640226
:1020B0007902B402C902DE02F10206031B033003F7
:1020C000450389075A036F03840399037E497F4CB4
:1020D00001A8FFF7AFFB7E4901A8FFF7ABFB217D0D
:1020E00001A8FFF7DFFB01A87A49FFF7A3FB207DDA
:1020F000FFF774FB14E47849744C01A8FFF79AFBCE
:10210000734901A8FFF796FB617D01A8FFF7CAFBA1
:1021100001A87049FFF78EFB607DE9E76F496B4CC2
:1021200001A8FFF787FB6A4901A8FFF783FBA17DA0
:1021300001A8FFF7B7FB01A86649FFF77BFBA07D6D
:10214000D6E76749614C01A8FFF774FB604901A815
:10215000FFF770FBE17D01A8FFF7A4FB01A85D4933
:10216000FFF768FBE07DC3E75E49584C01A8FFF725
:1021700061FB574901A8FFF75DFB217E01A8FFF72E
:1021800091FB01A85349FFF755FB207EB0E7564964
:102190004E4C01A8FFF74EFB4D4901A8FFF74AFB43
:1021A000617E01A8FFF77EFB01A84A49FFF742FBC9
:1021B000607E9DE74D49454C01A8FFF73BFB444934
:1021C00001A8FFF737FBA17E01A8FFF76BFB01A871
:1021D0004049FFF72FFBA07E8AE745493B4C01A809
:1021E000FFF728FB3A4901A8FFF724FBE17E01A88D
:1021F000FFF758FB01A83749FFF71CFBE07E77E7A4
:102200003C49324C01A8FFF715FB314901A8FFF703
:1022100011FB217F01A8FFF745FB01A82D49FFF71E
:1022200009FB207F64E73449284C01A8FFF702FB33
:10223000274901A8FFF7FEFA617F01A8FFF732FBEB
:1022400001A82449FFF7F6FA607F51E72B491F4C9C
:1022500001A8FFF7EFFA1E4901A8FFF7EBFAA17FEB
:1022600001A8FFF71FFB01A81A49FFF7E3FAA07FB7
:102270003EE72349154C01A8FFF7DCFA144901A8F1
:10228000FFF7D8FAE17F01A8FFF70CFB01A811497D
:10229000FFF7D0FAE07F2BE71A490C4C01A8FFF7B3
:1022A000C9FA0B4901A8FFF7C5FA94F8201001A854
:1022B000FFF7F8FA01A80749FFF7BCFA94F82000E5
:1022C00016E700BF186100082C5F0008000000201E
:1022D000295F00087B5E0008305F0008355F00085A
:1022E0003C5F0008445F00084B5F0008565F000831
:1022F000615F00086A5F0008735F00087C5F000888
:10230000855F00088F5F0008A249A34C01A8FFF772
:1023100091FAA24901A8FFF78DFA94F8211001A8BB
:10232000FFF7C0FA01A89E49FFF784FA94F821004C
:10233000DEE69C49984C01A8FFF77CFA974901A872
:10234000FFF778FA94F8221001A8FFF7ABFA01A87A
:102350009349FFF76FFA94F82200C9E692498E4C30
:1023600001A8FFF767FA8D4901A8FFF763FA94F80F
:10237000231001A8FFF796FA01A88949FFF75AFA36
:1023800094F82300B4E68949834C01A8FFF752FA78
:10239000824901A8FFF74EFA94F8241001A8FFF72C
:1023A00081FA01A87E49FFF745FA94F824009FE6D8
:1023B0007F49794C01A8FFF73DFA784901A8FFF75A
:1023C00039FA94F8251001A8FFF76CFA01A87449AE
:1023D000FFF730FA94F825008AE676496E4C01A89A
:1023E000FFF728FA6D4901A8FFF724FA94F82610A0
:1023F00001A8FFF757FA01A86949FFF71BFA94F8FB
:10240000260075E66C49644C01A8FFF713FA63498E
:1024100001A8FFF70FFA94F8271001A8FFF742FA76
:1024200001A85F49FFF706FA94F8270060E66349C0
:10243000594C01A8FFF7FEF9584901A8FFF7FAF92E
:1024400094F8281001A8FFF72DFA01A85449FFF7C6
:10245000F1F994F828004BE659494F4C01A8FFF7D1
:10246000E9F94E4901A8FFF7E5F9618D01A8FFF7E9
:1024700019FA01A84A49FFF7DDF9608D38E651499C
:10248000454C01A8FFF7D6F9444901A8FFF7D2F956
:10249000A18D01A8FFF706FA01A84149FFF7CAF983
:1024A000A08D25E648493C4C01A8FFF7C3F93B49FC
:1024B00001A8FFF7BFF9E18D01A8FFF7F3F901A823
:1024C0003749FFF7B7F9E08D12E64049324C01A8D1
:1024D000FFF7B0F9314901A8FFF7ACF9218E01A847
:1024E000FFF7E0F901A82E49FFF7A4F9208EFFE5D8
:1024F0003749294C01A8FFF79DF9284901A8FFF7A2
:1025000099F9618E01A8FFF7CDF901A82449FFF7D9
:1025100091F9608EECE52F491F4C01A8FFF78AF96D
:102520001E4901A8FFF786F994F8341001A8FFF7B7
:10253000B9F901A81A49FFF77DF994F83400D7E5F5
:102540002549154C01A8FFF775F9144901A8FFF7B3
:1025500071F994F8351001A8FFF7A4F901A8104902
:10256000FFF768F994F83500C2E51C490A4C01A848
:10257000FFF760F9094901A8FFF75CF994F83610F4
:1025800001A8FFF78FF901A80549FFF753F994F85F
:102590003600ADE5995F000800000020295F0008C3
:1025A0007B5E0008A35F0008AD5F0008B75F00080E
:1025B000C25F0008CC5F0008D65F0008E05F00083B
:1025C000EA5F0008F45F0008FE5F0008086000088A
:1025D000136000081E6000082960000834600008CD
:1025E000A249A34C01A8FFF725F9A24901A8FFF7CA
:1025F00021F994F8371001A8FFF754F901A89E4972
:10260000FFF718F994F8370072E59C49984C01A837
:10261000FFF710F9974901A8FFF70CF994F8381063
:1026200001A8FFF73FF901A89349FFF703F994F8D0
:1026300038005DE592498E4C01A8FFF7FBF88D4903
:1026400001A8FFF7F7F8618F01A8FFF72BF901A8A0
:102650008949FFF7EFF8608F4AE58A49844C01A861
:10266000FFF7E8F8834901A8FFF7E4F894F83C1075
:1026700001A8FFF717F901A87F49FFF7DBF894F8E5
:102680003C0035E580497A4C01A8FFF7D3F8794939
:1026900001A8FFF7CFF894F83D1001A8FFF702F961
:1026A00001A87549FFF7C6F894F83D0020E5774981
:1026B0006F4C01A8FFF7BEF86E4901A8FFF7BAF802
:1026C00094F83E1001A8FFF7EDF801A86A49FFF75A
:1026D000B1F894F83E000BE56D49654C01A8FFF791
:1026E000A9F8644901A8FFF7A5F894F83F1001A8DC
:1026F000FFF7D8F801A86049FFF79CF894F83F006D
:10270000F6E464495A4C01A8FFF794F8594901A826
:10271000FFF790F8B4F8401001A8FFF7C3F801A83C
:102720005549FFF787F8B4F84000E1E45A49504CA6
:1027300001A8FFF77FF84F4901A8FFF77BF894F84D
:10274000421101A8FFF7AEF801A84B49FFF772F854
:1027500094F84201CCE45149454C01A8FFF76AF8CE
:10276000444901A8FFF766F894F8431101A8FFF760
:1027700099F801A84049FFF75DF894F84301B7E4E0
:1027800047493B4C01A8FFF755F83A4901A8FFF724
:1027900051F894F8441101A8FFF784F801A83649CC
:1027A000FFF748F894F84401A2E43E49304C01A8F0
:1027B000FFF740F82F4901A8FFF73CF894F84511BE
:1027C00001A8FFF76FF801A82B49FFF733F894F839
:1027D00045018DE4032C40F0458433490398FFF70D
:1027E0000BF8292800F23E84DFE810F02A0062008E
:1027F00077008C00A100B600CB00E000F5000A01D4
:102800001F0134014901600176018C01A201B80168
:10281000F4010B02220239024F0265027B0291028F
:10282000A702BE02D502EC02020319032F034603DE
:1028300082039903B003C703DD03F30309041E04F5
:1028400004986946FEF7E7FF002800F00B84084C67
:10285000009B237502F098FC01A81449FEF7EAFFDB
:10286000044901A8FEF7E6FF39E400BF3F60000815
:1028700000000020295F00087B5E00084A60000815
:1028800056600008616000086B6000087560000811
:102890007F6000088A6000089A600008A160000854
:1028A000A8600008AC600008186100082C5F0008F0
:1028B00004986946FEF7AFFF002800F0D383B24CBE
:1028C000009B637502F060FC01A8B049FEF7B2FFFF
:1028D000AF4901A8FEF7AEFF16E404986946FEF77B
:1028E0009AFF002800F0BE83A74C009BA37502F05E
:1028F0004BFC01A8A749FEF79DFFA54901A8FEF7DB
:1029000099FF14E404986946FEF785FF002800F05B
:10291000A9839D4C009BE37502F036FC01A89E49FB
:10292000FEF788FF9A4901A8FEF784FF12E4049895
:102930006946FEF770FF002800F09483924C009BDC
:10294000237602F021FC01A89449FEF773FF904919
:1029500001A8FEF76FFF10E404986946FEF75BFFDD
:10296000002800F07F83884C009B637602F00CFC0B
:1029700001A88B49FEF75EFF854901A8FEF75AFFC3
:102980000EE404986946FEF746FF002800F06A83CB
:102990007D4C009BA37602F0F7FB01A88149FEF76E
:1029A00049FF7B4901A8FEF745FF0CE404986946FE
:1029B000FEF731FF002800F05583734C009BE3764F
:1029C00002F0E2FB01A87849FEF734FF704901A844
:1029D000FEF730FF0AE404986946FEF71CFF002862
:1029E00000F04083684C009B237702F0CDFB01A8E8
:1029F0006E49FEF71FFF664901A8FEF71BFF08E4BA
:102A000004986946FEF707FF002800F02B835E4C10
:102A1000009B637702F0B8FB01A86549FEF70AFF47
:102A20005B4901A8FEF706FF06E404986946FEF735
:102A3000F2FE002800F01683534C009BA37702F0AF
:102A4000A3FB01A85B49FEF7F5FE514901A8FEF77B
:102A5000F1FE04E404986946FEF7DDFE002800F06C
:102A60000183494C009BE37702F08EFB01A8524999
:102A7000FEF7E0FE464901A8FEF7DCFE02E40498FA
:102A80006946FEF7C8FE002800F0EC823E4C009B31
:102A900084F8203002F078FB01A84849FEF7CAFE0E
:102AA0003B4901A8FEF7C6FEFFF7FFBB0498694645
:102AB000FEF7B1FE002800F0D582334C009B84F86D
:102AC000213002F061FB01A83D49FEF7B3FE304919
:102AD00001A8FEF7AFFE20E404986946FEF79BFECE
:102AE000002800F0BF82284C009B84F8223002F0BE
:102AF0004BFB01A83349FEF79DFE254901A8FEF7CF
:102B000099FE1FE404986946FEF785FE002800F050
:102B1000A9821D4C009B84F8233002F035FB01A8EC
:102B20002949FEF787FE1A4901A8FEF783FE1EE435
:102B300004986946FEF76FFE002800F09382124C5D
:102B4000009B84F8243002F01FFB01A81F49FEF708
:102B500071FE0F4901A8FEF76DFE1DE40498694659
:102B6000FEF759FE002800F07D82074C009B84F898
:102B7000253002F009FB01A81549FEF75BFE044968
:102B800001A8FEF757FE1CE400000020305F00089B
:102B9000295F0008355F00083C5F0008445F0008BB
:102BA0004B5F0008565F0008615F00086A5F00081D
:102BB000735F00087C5F0008855F00088F5F000876
:102BC000995F0008A35F0008AD5F0008B75F0008C9
:102BD000C25F000804986946FEF71DFE002800F059
:102BE0004182B14C009B84F8263002F0CDFA01A856
:102BF000AE49FEF71FFEAE4901A8FEF71BFEFFF728
:102C0000F5BB04986946FEF706FE002800F02A820C
:102C1000A54C009B84F8273002F0B6FA01A8A5491C
:102C2000FEF708FEA24901A8FEF704FEFFF7F3BB7A
:102C300004986946FEF7EFFD002800F013829A4CD5
:102C4000009B84F8283002F09FFA01A89A49FEF709
:102C5000F1FD974901A8FEF7EDFDFFF7F1BB0498E0
:102C60006946FEF7D8FD002800F0FC818E4C009BE1
:102C7000638502F089FA01A89049FEF7DBFD8C49D3
:102C800001A8FEF7D7FDFFF7F0BB04986946FEF7F1
:102C9000C2FD002800F0E681834C009BA38502F072
:102CA00073FA01A88649FEF7C5FD814901A8FEF720
:102CB000C1FDFFF7EDBB04986946FEF7ACFD0028A7
:102CC00000F0D081784C009BE38502F05DFA01A80A
:102CD0007C49FEF7AFFD764901A8FEF7ABFDFFF793
:102CE000EABB04986946FEF796FD002800F0BA8119
:102CF0006D4C009B238602F047FA01A87249FEF74B
:102D000099FD6B4901A8FEF795FDFFF7E7BB049815
:102D10006946FEF780FD002800F0A481624C009B0C
:102D2000638602F031FA01A86849FEF783FD604925
:102D300001A8FEF77FFDFFF7E4BB04986946FEF7A4
:102D40006AFD002800F08E81574C009B84F83430D7
:102D500002F01AFA01A85E49FEF76CFD544901A879
:102D6000FEF768FDFFF7E0BB04986946FEF753FDE8
:102D7000002800F077814C4C009B84F8353002F03D
:102D800003FA01A85349FEF755FD494901A8FEF78A
:102D900051FDFFF7DEBB04986946FEF73CFD0028B5
:102DA00000F06081404C009B84F8363002F0ECF972
:102DB00001A84949FEF73EFD3D4901A8FEF73AFD4D
:102DC000FFF7DCBB04986946FEF725FD002800F0FC
:102DD0004981354C009B84F8373002F0D5F901A8C1
:102DE0003E49FEF727FD324901A8FEF723FD00E426
:102DF00004986946FEF70FFD002800F033812A4C45
:102E0000009B84F8383002F0BFF901A83449FEF77E
:102E100011FD274901A8FEF70DFDFFF7FFBB049840
:102E20006946FEF7F8FC002800F01C811E4C009B50
:102E3000638702F0A9F901A82A49FEF7FBFC1C49A7
:102E400001A8FEF7F7FCFFF7FEBB04986946FEF702
:102E5000E2FC002800F00681134C009B84F83C3013
:102E600002F092F901A82049FEF7E4FC104901A8FC
:102E7000FEF7E0FCFFF7FABB04986946FEF7CBFCCF
:102E8000002800F0EF80084C009B84F83D3002F0F1
:102E90007BF901A81549FEF7CDFC054901A8FEF70D
:102EA000C9FCFFF7F8BB00BF00000020CC5F0008A2
:102EB000295F0008D65F0008E05F0008EA5F0008AD
:102EC000F45F0008FE5F0008086000081360000857
:102ED0001E60000829600008346000083F60000898
:102EE0004A60000856600008616000086B600008D6
:102EF00004986946FEF78FFC002800F0B3807B4CF5
:102F0000009B84F83E3002F03FF901A87849FEF7B3
:102F100091FC784901A8FEF78DFCFFF7D1BB04981E
:102F20006946FEF778FC002800F09C806F4C009BFF
:102F300084F83F3002F028F901A86F49FEF77AFCC7
:102F40006C4901A8FEF776FCFFF7CFBB04986946F1
:102F5000FEF761FC002800F08580644C009BA4F81B
:102F6000403002F011F901A86449FEF763FC6149A1
:102F700001A8FEF75FFCFFF7CDBB049960484FF452
:102F8000807202F07DFC02F0FFF801A85D49FEF7B7
:102F900051FC01A85749FEF74DFC594901A8FEF71D
:102FA00049FCFEF71BBD04986946FEF734FC002877
:102FB00058D04E4C009B84F8423102F0E5F801A84D
:102FC0005149FEF737FC4B4901A8FEF733FCFFF7E8
:102FD000B6BB04986946FEF71EFC002842D0434C5D
:102FE000009B84F8433102F0CFF801A84749FEF76F
:102FF00021FC404901A8FEF71DFCFFF7B5BB049872
:103000006946FEF708FC68B3384C009B84F84431ED
:1030100002F0BAF801A83E49FEF70CFC354901A8B8
:10302000FEF708FCFFF7B5BB04986946FEF7F3FB13
:10303000C0B12E4C009B84F8453102F0A5F801A8E0
:103040003449FEF7F7FB2B4901A8FEF7F3FBFFF726
:10305000B5BB012C06D102F0F3F9FEF7BFFB002847
:103060007EF45EAC2C49FEF75CBC012CFAD102F078
:1030700033FAF2E7A31E012BF4D81C4B032C93F870
:103080004231009304D00099039802F049FAE6E730
:1030900004986946FEF7BFFB0028E3D0009B013B84
:1030A000632BF0D9DEE7022CDCD103986946FEF7EA
:1030B000B2FB0028D6D0009B03F5FA62B2F57A6F16
:1030C000D0D8164A1360164B00221A70FEF728BC9F
:1030D000012CC7D1134B1A68002ABCBF00221A600A
:1030E0001A68114B1A60FEF71BBC00BF00000020DD
:1030F00075600008295F00087F6000088A6000088A
:1031000042000020946000089A600008A160000856
:10311000A8600008AC600008B46000081007002038
:103120009806002048010020800100204FF08043D5
:10313000114A0021C3F82014C3F80C14C3F8041476
:1031400051640E4911652021916440F2A3515164EC
:103150004FF0FF32C3F82C2444210122C3F8142479
:10316000C3F808143321C3F81814C3F820244FF40B
:103170000072C3F80C2470470000024028020020AF
:1031800008B50D4B1B780BB1FFF7D0FF0B4B00229E
:103190005A644FF080438522C3F80024084A1288FD
:1031A000C3F82C246FF001010122C3F81424C3F8E2
:1031B0001014C3F80C2408BD68020020000002406F
:1031C000240200204FF0804370B5D3F80C1402297C
:1031D00048D0042900F0AF80012918D159485A4C31
:1031E0006FF001022568C3F810240268AA4225DAAC
:1031F00056490E68731C0B6056B9554B9A5C554B7B
:103200001A604FF0FF334FF08042C2F8343470BD83
:10321000092B07DC4F490A6802F001035210013BF9
:103220000A60F0E70132954202BF00230360236089
:103230004FF0000318BF02600B60E4E74422C3F8BC
:1032400008243022C3F820246FF00402C3F81024AD
:103250000422C3F80C2440F24A52C3F83424C3F8C1
:103260001414D4E76FF00202C3F81024374C394A23
:103270004FF09043D3F810142368581C01F010014C
:1032800020603BB919B1344B8021C3F8001C0023E6
:103290001360BCE70928136805DC5B100029F7D030
:1032A00043F08003F4E72748026819B140F2FF3188
:1032B0008A4203D128498025C1F8005C4FF0804143
:1032C0006FF00405C1F810540425C1F80C54082B04
:1032D0004FF00001216001D07F2B04D1002A96D04D
:1032E000013A026093E7551C19490560022D8B5481
:1032F00006D10A7822B94A78FF2A01D102F01EFCD1
:103300000A2B84D1002404604C551148FEF7D8FAEA
:103310000D4B186000283FF47AAF4FF08043012234
:10332000C3F80844C3F83444C3F81424C3F8202471
:10333000C3F80C246BE76FF00602C3F810240222D6
:10334000F6E700BF6C02002078060020840600200B
:1033500070020020100200200020004010B4424AF9
:103360004FF0804392F82820D3F83434002A65D0F7
:10337000A3F5A542013A40F2DE618A4231D9A3F5B4
:103380009642013A40F23E618A422AD9A3F525527B
:10339000013A40F26E318A4223D9A3F51652013A1E
:1033A00040F21E318A421CD9A3F5F052013A40F294
:1033B0007E218A4215D9A3F59652013AB2F5C77F0C
:1033C0000FD96FF470601A18B2F59F7F09D96FF4A6
:1033D00034615A18EE2A04D96FF4F0629A189E2AC2
:1033E0002CD8224A22484AF6AA211160214903F525
:1033F000FA7292FBF1F24FF47A7101FB02331E492B
:103400000A68134402680B600132026012F0030282
:1034100027D11A480468A342194C07DD5B42236098
:103420000A604FF0FF3010BC01F03EBE2468A3429A
:1034300004DA5B4203600A600120F4E7114B124A90
:103440001A604FF0804349F29122C3F818243122C8
:10345000C3F820246FF00402C3F810240422C3F838
:103460000C2410BC704700BF00000020003000405A
:103470008006002018FCFFFF880600209006002030
:103480009406002074060020313600084FF0804377
:10349000F0B4D3F8102412F001023BD06FF0010217
:1034A000C3F810244FF09042D2F8102412F010020A
:1034B00003D14E4B1A60F0BC70474D490A68013287
:1034C0000F2A0A60F7DD4B4A4B4911600022442164
:1034D000C3F82024C3F8081443F27821C3F8181461
:1034E0003021C3F820146FF00401C3F81014042134
:1034F000C3F80C14C3F8282440F69322C3F82C24F4
:1035000040F24A52C3F834240122C3F81424C3F809
:103510000024D0E73548D3F834140468651C0560EE
:10352000002CC8D0354E4CF6CC473760D3F8286411
:103530000C4606B3B1F5FA6F05DD2E4B304A1A6022
:10354000F0BCFFF70BBFD3F82814672908BF0C2283
:10355000C3F828240122C3F8142400230360AAE737
:1035600064100139812CFBDC264B1A688A4204D096
:1035700019600123F2E70221F4E700299BDB032D08
:1035800099DD1C4B204A1A60204B214A21481A60C1
:10359000214A884002EB6003B3FBF0F31F48013B74
:1035A0009BB203801E4800FA01F102EB6102B2FBFC
:1035B000F1F21C49013A0A804FF080420021C2F822
:1035C00020144421C2F808143321C2F81814012130
:1035D000C2F80C14C2F82C34134BC2F8141402F2C3
:1035E0003442DA64114A1A6565E700BF7C060020A0
:1035F0001402002074060020C5310008003000408D
:103600005D33000820020020D1360008700600203B
:1036100041370008F049020000EA32062402002087
:10362000D8B8050026020020000002402802002031
:103630004FF0804313B5D3F83424D3F83804B2F5EF
:10364000FA6F0ADBA0F11C03042B08D81C4B4AF6C6
:10365000AA221A601B4B01221A7002B010BDA0F5FD
:103660004873B3F5AF6FF8D8154B174C4AF6AA223A
:103670001A6094F82430BBB1A18DA1F132029042BE
:1036800009DA0023618D0093A3F5FA6301F03CFD94
:103690000E4B1860E1E7323188420DDD4FF4FA63DA
:1036A00000930023E28DF1E7618D3231884205DD20
:1036B0004FF4FA620092F5E70020E9E71846E7E7E1
:1036C0000030004005070020000000201007002007
:1036D0004FF08043D3F80C24D1072BD5D3F8102416
:1036E000D20727D56FF00102C3F81024D3F82024A5
:1036F00052B90122C3F820244FF090430E4AD3F868
:10370000103403F0100313700C4B20229A6440F223
:10371000A3525A644FF080434FF0FF32C3F82C2479
:103720000122C3F814248122C3F800244FF400724C
:10373000C3F80C24704700BF68020020000002405C
:10374000B5494A6C12F01002F8B548D0B348FFF7FB
:10375000EDFC02686AB9B24B19684FF6807311B17B
:103760008B42A8BF0B46B3F5007F2EDA43EA422313
:103770000360036819011A461B1129D1D24302F0D4
:103780000F02A84E0A4319468C0042FA04F505F0D0
:103790000F050C44755D013105FA04F4042943EA70
:1037A0000403F1D1A04C13224FF0FF3143FA02F58C
:1037B000ED0748BFC943013A24F8021FF6D29B4ADD
:1037C00013683BB900230360F8BD5B100132CAE700
:1037D0005A40D1E7013B1360002BF3D0F4E7944C3F
:1037E000237873B34FF080437820C3F82024C3F8C4
:1037F0000824C3F81824C3F818040820C3F80404E4
:1038000089484A6408651720886440F293504864E8
:10381000C3F8342472B6D3F82424C2F542620F32BE
:10382000132AB8BF1322C3F82C240122C3F814248E
:10383000D3F814147F490988C3F82C14C3F8202442
:1038400062B67D4B7D481988002201318D101346E8
:1038500047885B00AF4202F10202A8BF43F00103B8
:10386000202A064618D1207819461A4609111CD17B
:1038700000B1D24312F00F0213D171494AF6AA20C7
:10388000086003F010015B1100F05D812F2B11DD4A
:10389000002900F05D8157E1B6888E4200F10400F6
:1038A000D6DBBDE8F840FFF76BBC4A40DEE7A3F18A
:1038B0002F025BE1002987D0594A1068002883D184
:1038C00060490A689A42604A1CBF0B601060136826
:1038D000092BDCBF013313600B68591E2E293FF6FC
:1038E00073AF01A050F821F0A5390008A5390008F0
:1038F000A5390008A5390008A5390008C93700080E
:10390000AB390008BB390008C9390008DB390008A9
:10391000C9370008E9390008FB3900085D3A00089A
:10392000C9370008C9370008C9370008C937000877
:10393000C9370008733A0008833A0008C9370008FD
:10394000C9370008C9370008C9370008C937000857
:10395000C9370008C9370008C9370008C937000847
:10396000C9370008C9370008C9370008C937000837
:10397000C9370008C9370008C9370008C937000827
:10398000C9370008913A0008BB3A0008E53A000838
:103990000F3B0008C9370008C9370008C9370008BD
:1039A000393B0008294A13700EE71368062B7FF491
:1039B0000BAF274B00229A7506E71368062B7FF49E
:1039C00003AF234B0122F6E71368062B7FF4FCAE0E
:1039D0001F4B002283F82420F6E61368062B7FF4A1
:1039E000F3AE1B4B0122F5E71368062B7FF4ECAE18
:1039F00001F026FD174B1860E6E61368062B7FF4EE
:103A0000E3AE154B01221A70044B4FF460621A604A
:103A1000064B0A22AEE000BF00000240C8060020AC
:103A2000D0060020C46100084C0100208C06002054
:103A30006802002026020020240200202802002024
:103A400000300040180200201C02002099060020CF
:103A50000000002080010020C40600201368062B0F
:103A60007FF4B2AE444B00221A70444B40F6FF6222
:103A7000CDE71368062B7FF4A7AE414B00221A70E6
:103A8000A2E61368062B7FF49FAE3D4B0122F6E7BA
:103A90001368062B7FF498AE3A4A137E5B08013315
:103AA0000F2B08D8082BB8BF082359001176073B05
:103AB000354A136088E60823F7E71368062B7FF47E
:103AC00083AE3049CA7E920801320C2A03D8062AF6
:103AD0001346B8BF0623DAB29000D200C8760A7740
:103AE000053BE5E71368062B7FF46EAE25490A22F5
:103AF00091F82030B3FBF2F30133DBB20B2B28BF7C
:103B0000002303EB8302520081F82020D0E71368E2
:103B1000062B7FF459AE1B490A2291F82130B3FBE2
:103B2000F2F30133DBB20B2B28BF012303EB83023B
:103B3000520081F82120BBE71368062B7FF444AEC6
:103B400001F0CAFC56E789B11049012008706BB139
:103B50000C4A92F82420002A3FF4A9AEB3F5836FF3
:103B6000ACBFA3F21743C3F12F035A00084B1A60EE
:103B7000084B00221A6027E6C4060020C806002071
:103B8000D50600200000002080010020050700204D
:103B90001007002018020020124B134A1A604FF041
:103BA00080434FF40042C3F844245422C3F808244D
:103BB0003122C3F8182403210122C3F82024C3F8BA
:103BC0000C146721C3F828144FF0FF31C3F82C14EC
:103BD0000421C3F80014C3F814248522C3F8002478
:103BE000704700BF740600208D340008014B1B682D
:103BF000184700BF74060020034B4FF400525A6070
:103C0000024B1B68184700BF0000024070060020EE
:103C1000014B01225A61704700100040B44BB54976
:103C20002DE9F0471E68B44DB44C2B68002E71D0BE
:103C30004FF0804201205663D662B14E5061327817
:103C400022B91BB13C2253433B3B2B600A782B68C3
:103C5000002A53D0013B002BD8BF4FF4B4732B6024
:103C600029684A1E772A4FDC01F1EF077731A54812
:103C7000A54B05689B7EC5F17805DB00AB42A8BF6C
:103C80002B4618468323C4F8003C41F2EC03C4F8E9
:103C90002C3C9E4B33F812204243D2113932C4F8E7
:103CA000342C33F8172033F8113042434343D211F8
:103CB000DB1139333932C4F8382CC4F83C3C812349
:103CC000C4F8003C3578BDB946F66803C4F8183C22
:103CD0006823C4F81C3C40F25553C4F8203C21230F
:103CE000C4F8143C4FF080432846DD60FDF7E4FC47
:103CF000874B1D6001233370BDE8F0870133B3F5B6
:103D0000B47FC8BF0123AAE7EF2AA1F17907ADDD8F
:103D1000F139ACE70F78002F00F08180013B002BD8
:103D2000D8BF06232B602B687A4A1A4403F001039C
:103D300012F8012C02EAD200D143BB4218BF04267C
:103D400010F0010301EAD2016ED06F4A527D002AC1
:103D500018BF052343F4805340F66802870771D5E6
:103D6000694F7F7D002F14BF5027102742F4C042B7
:103D70003B43400771D56449497D002914BF4FF486
:103D8000A0614FF480710B4346F66801624FC4F89E
:103D9000182C3868C4F81C1CC4F8203CFDF78CFCB7
:103DA0003E605E4FDFF868913868DFF874815D4EE1
:103DB000B0F57A6F5CDD5C4B4FF47A621A600023D9
:103DC000C8F800303368632B4FF0000270DCC4F891
:103DD000402C4FF080434FF4E242DA6185221A60B2
:103DE0004FF0804300221A611122DA602B684F4A9B
:103DF0003968013B42F82310D9F80030052B7FF7D2
:103E00007BAFD2E900310B4491680B44D1680B447D
:103E1000116952690B441344DB1033606CE70133C2
:103E2000062BC8BF01237DE7CB075DBF46F0010627
:103E300041F2040340F6480241F2040348BF40F651
:103E400058028BE78F0743F040034EBF42F4A04275
:103E500042F4804246F002068BE7490743F4806350
:103E60005ABF46F0030646F6480146F658018DE76C
:103E7000D8F800300133062BC8F80030A2D1DFF8A3
:103E8000A8A0DAF80030181A01F08EFC3B68B0EBFD
:103E9000630F09DD264A0023C9F80030137044F689
:103EA00020633B60234B33603B68CAF8003086E7F1
:103EB000C72B06DCC4F8402C4FF080434FF411426E
:103EC0008BE7B3F57A7F06DAC4F8402C4FF08043D5
:103ED0004FF4414281E7B3F5FA6F4FF080432BDA9C
:103EE000C4F8402C4FF44142DA6140F2851276E783
:103EF000F8060020F5060020FC0600200020014006
:103F0000EC060020C006002000000020A45B000892
:103F100000070020A6630008E8060020DC06002059
:103F2000B4060020D0060020240700209C060020B4
:103F3000D406002000E1F5054FF40072C4F8402CCF
:103F40004FF44142DA6140F2852248E738B501F08A
:103F5000D5FA1749174A0B68174C5BB113784BB168
:103F600023683C201D3393FBF0F30133062BC8BFBD
:103F70000123236000230B601370104B104D1B783E
:103F80006BB1FFF74BFE2123C5F8143C0020FDF771
:103F900093FB0C4B22681A600023236038BD46F661
:103FA0006803C5F8183C6823C5F81C3CEBE700BF64
:103FB000F8060020EC060020FC060020E0060020A9
:103FC00000200140E4060020144BD3F80C2C92068C
:103FD00023D5D3F8182CD3F81C1C02F0700040280D
:103FE00008BF22F0700202F4E040B0F5804F01F00B
:103FF000700008BF22F4E0424028C3F8182C08BF24
:1040000021F070012022C3F81C1CC3F8142C6FF09F
:104010002002C3F8102CFFF701BE704700200140BA
:104020004FF0804310B5DA681969D00712D5C90777
:1040300010D56FF001021A610022DA60214B1A607C
:10404000214B1A70214B49F640421A60204B214AFD
:104050001A6010BDD306FCD51C484FF0804302689F
:104060001B6CB3EB620FF4DB02EB4202B3EBA20F6B
:1040700002DBB3EB620F22DD15490968B1F5FA6F77
:10408000ACBF002101211344134A0F4C127E217052
:104090009B105A430360A3EB62135B104FF0804206
:1040A000012BB8BF01235363012353610023D36065
:1040B000044A1368052BDCBF01331360C9E70021F4
:1040C000E1E700BF00070020D4060020DC06002046
:1040D000D006002000E1F5050000002073B5014680
:1040E0003F48404C164602689B1A67D40123237050
:1040F0000A223D4801F01AF83C4A831023EAE37390
:10410000136000210A220546394801F00FF83949A9
:10411000394A831023EAE373714313604914072279
:104120000446364801F002F8354B0422186000219D
:10413000344800F0FBFF344B344918600B681844D6
:10414000334B08601A68C2F3090252B9314E0A6053
:10415000336803EBA0235B20336043432E48DB131B
:1041600003602E4E96F83C3083B196F83D20012A2C
:104170004FEA83032BD0022A2BD032B35B4223EACF
:10418000E373274A3C2BA8BF3C231360254B1B78C5
:1041900093B106992448052200F0C8FF96F827300D
:1041A0004FF4FA62009203EB83039B00728E318E10
:1041B00000F0AAFF1D4B186002B070BD2478002CDF
:1041C00096D102EB6302026092E7EB1AD7E7E31A9B
:1041D000D5E7A542ACBFC3EB0503C3EB0403CEE7B1
:1041E00098010020F40600208C0100200807002020
:1041F00090010020E43202000C070020940100200E
:104200002807002088010020BC060020D8060020D6
:1042100018070020F0060020B8060020000000204B
:10422000C00600209806002084010020100700200E
:104230004FF0E0234FF08052C3F8042D0022C3F862
:10424000102D094A13780133DBB2137013F00F03FA
:1042500009D106490A6801320A60054909688A429B
:1042600004BF044A13707047140700201807002089
:10427000200700201C07002038B50C4672B6074BFB
:10428000074D1B681844074B186001232B7062B65A
:104290002B7803B938BDA047FAE700BF1807002004
:1042A0001C070020200700202DE9F047204C237830
:1042B0008AB053B11F4A013B92F843111E4A52F88B
:1042C000230001F02DF9002323701C4F3B68002BC5
:1042D0001BDB184A92F842616A46192EB8BF1926AC
:1042E000002490460A20B3FBF0F100FB113342F8A2
:1042F000043B01340B460029F5D1DFF84490DFF888
:1043000044A023465D1E1BB93D600AB0BDE8F0879E
:104310009C4204D049464FF4FA70FFF7ADFF58F8BD
:10432000253031465AF8230001F0FAF82B46E9E728
:1043300099060020000000204C6200088001002047
:10434000113C0008AC63000838B5114C23782BB140
:10435000104B1D7815B900F0D1FD25700E4B1B7860
:104360001A0713D1FDF7BCF90C4B1B68DB0601D112
:1043700000F0FCFD0A4B93F845010A4B1A68824293
:1043800004D01860BDE8384000F08CBE38BD00BFD6
:10439000050700200407002014070020180700204C
:1043A000000000207C01002008B5012000F07AFE0A
:1043B0000D4B8022C3F8142CA3F5883342F69F02DC
:1043C0009A6242F20F72DA6201225A616FF00102C0
:1043D0001A6109221A601A68D207FCD4034B8022A2
:1043E000C3F8002CFEE700BF002001400020004081
:1043F0002DE9F04FAC48AD4AAD4CAE49AE4E95B04C
:10440000121A01F003FA00F0BFFEE37D0693AB4BF6
:1044100094F823201A7094F82730A94A03EB8303F9
:104420009B001360A74B94F836201A70FDF748F8EC
:1044300000F036FE00F035FE00F0C6FCFFF7ACFBE6
:1044400048F63903C6F8443C41F2EC03C6F82C3C6C
:104450008123C6F8003C3523C6F8043C4FF0804366
:104460000C229A6200250422DD621A6001225A6140
:1044700085221A608021FE2001F074FB4FF0E023BA
:1044800041F663125A6107229D611A6194F83F3028
:104490008D4A07931378002B00F0E580079B43B902
:1044A0008A4B1B684FF4DC7203F2B71393FBF2F3F1
:1044B0000793874B5D6A4FF0807215F0C04F5A62C8
:1044C0001BD194F842307E2B40F0CF80814801F020
:1044D0006FF920EAE07164297F48A8BF642101F0E8
:1044E000DDF894F83E3043B17C4B079A7C491A6062
:1044F000FA20FFF7C1FEFFF7D7FE237D0BB96C0052
:104500001ED5784C6E4D42F69F03A36240F6C3134E
:10451000E3620423236001270523676123606FF0B2
:10452000010323612F602369D80740F1A480002391
:104530002B6023605E4B6C4893F8421100F0F0FF53
:10454000FFF704FD1422002109A801F06DF93223C0
:10455000089314224FF47A7300210FA80A9301F0F4
:1045600063F94FF4C8730E934FF416734FF0000ABB
:1045700010934F4DCDF810A00223D3465746039316
:10458000D046D146049AE87E584BB3FBF0F305932E
:1045900040F6B8339A42697E18BF494B01EB81015E
:1045A00014BF1C680024890014BF4FF00A0C4FF0A0
:1045B000000CB8F1000F08BF4FF00009002C40F0CC
:1045C0009F80039B95F82320012B08BF02230393B0
:1045D0003A4B1978914208D0069931B91A70B8F15E
:1045E000000F02D1FFF7B2FC344B1B78002B4BD0ED
:1045F0003F4B95F822001C68C4F164048442A8BFB4
:1046000004464FF000082D4B1B78002B40F03D82F4
:10461000B8F1000F00F03B826B7D002B0CBF002334
:104620003923069A002A00F03482059A9C3A0092B7
:1046300000214FF4FA62204600F066FD8323C6F89D
:10464000003C059BC6F82C3C8123C6F8340CC6F808
:10465000380CC6F83C0CC6F8003CB8F1000F00F06E
:104660004882A14695E030BF14E794F842112148F2
:1046700000F056FF35E730BFFFF716FE2B68002B22
:104680003FF451AF67614EE71B4A1268052A05DD0A
:104690001A4A1268B2F5487F80F2EB8195F8224001
:1046A00004EB8404A400ACE70000002048010020D3
:1046B000000000200010000800200140E00600205B
:1046C0001007002004070020F4060020280700201F
:1046D0000010024043000020E8670008800100202D
:1046E000113C000800100040D46100084096010011
:1046F000C00600204200002000070020CC06002059
:1047000080F2DA8095F82430022B40F0BE80039BC3
:10471000022B40F0BD80784BAA7D95F825001B78D0
:104720000438002A08BF83F00103744A4443A410EC
:104730001370DFF8CC81D8F80030002B40F0C58032
:10474000CCF100030B44A34280F2C180A87F6B7FB1
:1047500000EB8000800003EB830300909B00204669
:104760004FF4FA62614400F0CFFC0446644B1B68CE
:10477000002B00F08081002C40F0DA80614A116843
:1047800039B12D214B4313605F4A92FBF3F35F4A2B
:1047900013605F4A13681BBB069B5A49002B00F04D
:1047A000858156486C7D0378002B00F0748140F2BF
:1047B000144C40F25443002C08BF6346582446F67C
:1047C000580CC6F818CCC6F81C4CC6F8203C21235F
:1047D000C6F8143C0378013313604FF416730B6072
:1047E00001234FF0E0220221C2F8101D30BF494AD8
:1047F000127812F00F0146D1049840F6B732904279
:1048000000F39B81079895F83E2042430A204243DB
:1048100041480068824240F39481049A0132049234
:104820006A8F002A00F08F813C49B1FBF2F23C49CB
:1048300005930968A2F54872891008A800F08AFC5F
:1048400007EB204727EAE777A02F059BA8BFA02703
:10485000B5F84020002A00F0788164214A433149AC
:10486000059309680EA800F075FC0BEBA02B2BEA52
:10487000EB7BBBF5FA6F059BA8BF4FF4FA6B059372
:10488000FFF712FD059B98467CE6032B7FF443AFB0
:1048900095F8222095F82630234902EB82029200F7
:1048A00003EB830300929B002046002200F02CFCC7
:1048B000012304460393A4E60F4AAB7D12785340CC
:1048C0000E4A13700023039333E763463AE7A1EBE4
:1048D0000C02698F69B1154BB3FBF1F300932046CD
:1048E0004FF47A63002100F00FFC0024C8F80000A8
:1048F0003CE74FF41173F1E7D5060020F5060020E0
:10490000F8060020D006002000879303CC06002084
:10491000FC0600201407002028070020002D31018C
:10492000DC060020BC06002030F8FFFF54581400BD
:1049300072B689490B7813B3884FDFF824C23B68FD
:104940009CF800C0581E3C2390FBF3F2BCF1000F12
:1049500000F0FD800132062A90FBF3FC03FB1C03F0
:1049600008BF00220133D8F8000043434FF08040D5
:1049700043637C4BC36201231A4443613A607A4B20
:1049800000271F60794BC8F800701F70784B0F70BC
:1049900049F64048C3F80080FFF740F962B6414647
:1049A00008A800F0D3FB4FF00108B946069B43B1BD
:1049B0006B4B6A4A1B78116801338B421CBF002382
:1049C00013606C4BA7EB0B000444186824EAE474F2
:1049D00088B1694B93FBF0F0684B2A7F186047F26F
:1049E0003051674BB3FBF2F34EF660220093059B08
:1049F00000F08AFB0590EB7F95F820205F484FF48C
:104A0000FA61009103EB83034FF47A714A439B00F0
:104A10000068002100F078FB5A4B1B686FF0180209
:104A2000534303F5FA639C42A8BF1C464F4B1B78C7
:104A30008442A8BF04460BBB95F82130DA1003F07E
:104A4000070353450AF1010AC8BF0132BAF1080F42
:104A500008BF4FF0000A4C4512DA434B1B68052B88
:104A60007FF7D1ADA9EB02094C453FF7CCAD4C46E1
:104A7000C9E51F469AE74FF0010897E70023DDE7F5
:104A800091444C45FFF6BFADF1E73923C9E54346F4
:104A9000C7E5059ACBE540F2411C40F24553002C96
:104AA00008BF6346682445F6680C8AE672B6364B42
:104AB0001B6813602E4B49F640471F60334B0B6059
:104AC000FFF7ACF82123C6F8143CD6F80C3C4FF0A5
:104AD000804243F03103C6F80C3C0124214B536360
:104AE000D362546162B6394608A800F02FFB069FD6
:104AF00076E61A4B1B68F3B172B6D6F80C3C23F07D
:104B00003103C6F80C3C4FF080430122C3F80C80FF
:104B1000C3F82C805A61FFF719FA134BC3F80080D1
:104B2000124B83F80080134BC3F80080134BC3F87B
:104B3000008062B64346A14653E6002B7FF470AE78
:104B4000DFE404916CE6174682E6934697E653430A
:104B50001B1A3C3307E700BFEC060020FC060020D0
:104B6000F5060020FFFF030000070020D406002008
:104B7000DC060020D006002000879303CC0600202E
:104B800040960100C0060020E406002000E1F50583
:104B9000C0F57F43CAB2F93330B59B1AC1F307227F
:104BA0009B1A064A04460D12062013711B12107040
:104BB00054709170D570537130BD00BF2C07002028
:104BC0000368134403EB2323DBB210B50360A2F1A7
:104BD0007D03012B064806D80B685C1C0C607D2405
:104BE000C45402F0DF020B685C1C0C60C25410BDA0
:104BF0002C07002037B500230C46054601A968465E
:104C00001022CDE90033FFF7DBFFEAB26846FFF779
:104C1000D7FFC5F307226846FFF7D2FFE2B2684626
:104C2000FFF7CEFFC4F307226846FFF7C9FFC4F3BE
:104C300007426846FFF7C4FF220E6846FFF7C0FF31
:104C4000009AD2436846D2B2FFF7BAFF019803B088
:104C500030BD0000042830B402464CD1274B1978EF
:104C6000042948D158785B884FF6FB7103448B4286
:104C700041D1234C94F837306FF00505591E00F0F0
:104C80000F0305FB0133013B052B34D8010909292A
:104C900007D00A290BD0082918BF0022104630BCC3
:104CA0007047184A32F8131030BCFFF771BF013B50
:104CB000042B04D8DFE803F0090B0E101200124B8E
:104CC0001B680A2128335943EEE7104BF8E7104BD5
:104CD0001968E9E70F4BFBE70F4BF9E794F8381039
:104CE0000E4B49081B6893FBF1F34FF6FF71994295
:104CF000A8BF1946D8E70022D0E700BF2C07002044
:104D000000000020D8630008080700200C070020DE
:104D100028070020BC060020B8060020CC06002092
:104D2000022810B438D11E4B1A787E2A34D11D497E
:104D30005A7891F8373002F01F02013B9A422BD18A
:104D4000194A1A481368062B04BF0023136013681E
:104D50005C1C30F813001460052B1DD8DFE803F04D
:104D600003080A0C1214124B196810BCFFF742BF5B
:104D7000104BF9E7104BF7E7104B1968CD23594357
:104D8000C912F2E70E4BEFE791F838300D4A5B0895
:104D9000116891FBF3F1E8E7002010BC704700BFF9
:104DA0002C0700200000002044070020E4630008D6
:104DB000080700200C07002028070020BC06002060
:104DC000B8060020CC060020244B40F28732C3F8FE
:104DD0000C28234A1178234A03291ED0042934D0F1
:104DE000022908D1204911600C21C3F814184FF48E
:104DF0000001C3F804181268184B52B3C822C3F854
:104E000008281D22C3F80028184B194A9A6319492B
:104E1000194ADA6359629A6270471849116040F280
:104E20000E71C3F80C181A21C3F814184FF40301BB
:104E3000C3F804184FF09041D1F80C3423F44053D8
:104E400043F40053C1F80C34D5E7FA21C3F80C1829
:104E5000D1E78822C3F808280922D3E700300140AF
:104E6000040700203C070020554C000800000240C9
:104E700024380140283801402C070020214D00082B
:104E800070B5164CD4F8006816F0400619D1082306
:104E9000C4F81838124D40F61803C4F82038686B6F
:104EA000104BC0F110001B68984750B14023C4F864
:104EB00020384923C4F800389123EE612862EB6161
:104EC00070BD064B084AC3F8002803F55043002282
:104ED0001A6310225A6381221A63F1E700300140FD
:104EE000000002403C0700200D000004024B20227D
:104EF0005A600022DA6170470000024038B5144D54
:104F0000EB69DB0723D4134B134C1B682922534353
:104F1000124A12682270124A1268A2701112114AC3
:104F200061701268227111120F4AE1701268A27149
:104F3000111261711A1509211B1320462372E271A7
:104F400000F0C2F80A2360722B629323EB6138BD34
:104F500000000240CC0600202C070020080700209B
:104F600028070020BC060020B806002038B5354BC5
:104F70001B78012B0FD0042B10D0334B1B78002B48
:104F800043D0324A1368591C1160032B57D8DFE80D
:104F900003F0323D424BFFF7B1FFEEE72C4DE869DD
:104FA00010F00100E9D12B4B2B4C1A682B4BA0724F
:104FB0001B68CD214A434B43C82121700A216170EF
:104FC0000821A170D114D2122271DA14DB12A3715C
:104FD000234B62711B68E1701A14E27109211A12E5
:104FE000A01C6372227200F07FF80C23E0722B6227
:104FF0009323EB61C1E71B4B1B7843F4007372B63C
:10500000194A116801B9136062B638BD174B1B7895
:1050100043F40063F3E70F4B1B6829225343C3F3A8
:10502000872343F48063EAE70C4B1B6829214B4339
:10503000C3F30733002143F4C0631160DFE70023AB
:10504000DDE700BF04070020C40600204007002061
:1050500000000240280700202C070020BC0600208A
:10506000B806002008070020C80600200C07002012
:105070000A4B01225A6103F58833D3F8102CD2076A
:105080000BD56FF00102C3F8102CD3F8342CD3F8F1
:105090003C1CC3F8341CC3F83C2C70470010004083
:1050A000704770477047000006490B68C3F3C4029D
:1050B000104480F3050023F0F80343EAC0030B60BB
:1050C000704700BF0010024010B5064A0346014475
:1050D00000208B4200D110BD13F8014B6040105CE2
:1050E000F7E700BF0A65000810B5064A0346014409
:1050F00000208B4200D110BD13F8014B6040105CC2
:10510000F7E700BF0A64000810B504468C42184651
:10511000029B0ADD9442BFBF641A1B1A5C43521AF9
:10512000AEBF184694FBF2F4001910BD00290BDB4A
:105130000368002BB8BF01FA02F319441341C91ADE
:10514000016041FA02F07047002070470023C0E977
:105150000431704730B5D0E903548A1A13196C42F0
:10516000A342B8BF2346AB424469A8BF2B46C0E95F
:1051700004310C1BD0E9001580686B4301FB02333E
:1051800000FB043030BD000030B5AC4B1C7DD87D39
:10519000221E18BF01221A755A7D111E18BF012147
:1051A0005975997D003918BF01219975011E18BFE5
:1051B0000121D975197E0129B8BF01211F29A8BF76
:1051C0001F211976597E59B1002A00F02681002846
:1051D00040F023810529B8BF05211929A8BF19214D
:1051E0005976997E1D7F0129B8BF01210F29A8BFDB
:1051F0000F219976D97E1029B8BF10213029A8BF78
:105200003021A942D976B8BF29466029A8BF6021BC
:105210001977597F9D7F0129B8BF01216429A8BF53
:105220006421A9425977B8BF29466429A8BF6421DF
:105230009977D97F93F823500129B8BF01216429B8
:10524000A8BF6421D97793F820106429A8BF6421EE
:1052500083F8201093F821100129B8BF0121642997
:10526000A8BF642183F8211093F822106429A8BFF5
:10527000642183F82210002D00F0D18012B1B0FA21
:1052800080F25209002A93F8245083F8232008BFA3
:105290000322AA42A8BF2A4683F8242093F8252097
:1052A000032AA8BF032283F8252093F826208A42E8
:1052B000B8BF0A46642AA8BF642283F82620002CBF
:1052C00093F8272014BF002164218A42A8BF0A4610
:1052D00083F8272093F82820003A18BF012283F88A
:1052E00028205A8DB2F5617FB8BF4FF4617240F249
:1052F0006C718A42A8BF0A46D98D5A8502F1C8044A
:10530000A142B8BF214640F63404A142A8BF2146BD
:105310009C8DD9856432A242A1F16401B8BF2246B6
:105320009142A8BF11461A8E9985B2F5486F598EE1
:10533000A8BF4FF448621A86C8328A42B8BF0A46EC
:1053400040F648518A42A8BF0A4693F836105A865A
:1053500004290C464FF00002A8BF042402299A86B3
:1053600083F836405DD193F83720012AB8BF012277
:10537000022AA8BF022283F8372093F8382022F0AF
:105380000102022AB8BF0222642AA8BF642283F85D
:1053900038205A8F5AB100284ED140F2DC518A424F
:1053A000B8BF0A4640F6AC518A42A8BF0A465A879F
:1053B00093F83C202AB13C2AB8BF3C228C2AA8BFD3
:1053C0008C2283F83C20002283F83D2093F83E2075
:1053D0002AB11C2AB8BF1C22262AA8BF262283F87D
:1053E0003E2093F83F20182AA8BF182283F83F20B8
:1053F00093F84221642AA8BF642283F8422193F8DB
:105400004321642A4FF00001A8BF642283F843219E
:10541000A3F84411A3F8401030BD0021E0E62A466D
:1054200030E70329A7D193F83720012AB8BF01221A
:105430001C2AA8BF1C229EE70022B8E7000000201B
:1054400038B51E4B1B680BB1002038BD1C4B1B78B8
:10545000002BF9D172B61B4B1B4A5A6002F18832FD
:105460005A604FF0FF32DA6002221A61174A5A611D
:1054700042221A61DA68D207FCD401221A61144B65
:105480001249144A0F481C4693420FD380230361EC
:1054900062B6C36813F0140FD6D10D490B48121B26
:1054A00000F0A4F9B0FA80F04009CEE733F8025BCF
:1054B00021F8025BC568ED07FCD4E5E7D0060020C3
:1054C0004807002000200240230167450010000823
:1054D000000000204801002008B572B605490648C2
:1054E0004FF4A37200F092F962B6BDE80840FFF7EE
:1054F000A7BF00BF6062000800000020074B44F215
:105500004002C3F8182C4022C3F81C2C40F244423D
:10551000C3F8202C2122C3F8142C7047002001402E
:105520002DE9F74F0F460A2201A9064600F06EFA50
:10553000019BB34246D0A0F10A0140F2DD32914214
:1055400000F29F801E4643F6982898FBF0F8002F43
:1055500000F097804C4B1868002840F09280DFF8EC
:105560002C9199F8001051BB494CDFF828A1012378
:1055700089F80030FFF7C2FF45F26803C4F8183C11
:105580006823C4F81C3C40F24553C4F8203C0C236B
:10559000C4F8283C8B46354615F8012BAAB90021E2
:1055A00041F2EC03C4F8281CC4F82C3CFFF7A6FF1A
:1055B00015F8010C89F80010B0FA80F0400903B02A
:1055C000BDE8F08F4FF07D08C1E7A2F16101062927
:1055D00021D8633A00210732072092FBF0F0C0EB9C
:1055E000C000121A520070782B4B042AC8BF02F177
:1055F000FF32232808BF0132594433F8122042FAFF
:1056000001F107F10502C4F82C1C08BFB51CC4F851
:10561000342C00220BE0A2F14101062902D8433AC2
:105620000121D8E75F2A1AD10022C4F8342C2123A3
:10563000C4F83C2C01A90A22C4F8143C284600F006
:10564000E5F9019AAA421AD0411E6229A7D8154647
:10565000514600FB08F0FEF70FFE2E469BE72B2A73
:1056600005D1BBF1000F9AD14FF0010BF5E72D2AC0
:1056700095D1BBF1000F92D04FF0000BEDE7012068
:10568000E6E700209BE700BFD00600204807002087
:105690000020014071500008F06300082DE9F84334
:1056A00002683B4B9A4271D1C368B3F1007F6DD160
:1056B0004369B3F1807F69D1002967D0354B1B68FE
:1056C000002B63D1344E3578002D5FD14FF00108A7
:1056D00086F80080FFF712FF304A314C45F268032C
:1056E000C2F8183C682740F24553C2F81C7CC2F847
:1056F000203C41F2EC03C2F8345CC2F83C5CC2F8D6
:105700002C3C2123C2F8143CA56203691DBA254B29
:1057100003EB5503B3FBF5F3013BE362C4F81480DC
:10572000C4F80080436885681BBA2DBA18446FF02E
:10573000010805444FF0830E4FF0810C2369DB070D
:10574000FCD52B1A002BC4F810801ADD10F9013B90
:10575000C2F800EC03F18009C3F17F0301FB09F9F2
:105760004B4307FB09F97B434FEA69395B1309F1A6
:1057700039093933C2F8349CC2F83C3CC2F800CC39
:10578000DCE700212160FFF7B9FE3170BDE8F88346
:105790002E736E64D00600204807002000200140D0
:1057A0000010004000EA32060028B8BF40427047AF
:1057B0000A22002100F02AB9931E222B10B50C46B4
:1057C00004D900230B701C46204610BD0A2A09D1BB
:1057D000002807DA2D230B7040420121214400F0FC
:1057E0001FF9F1E70021F9E7FFF7E6BF10B501392E
:1057F0000244904201D1002005E0037811F8014FE6
:10580000A34201D0181B10BD0130F2E70A449142B7
:1058100000F1FF3300D1704710B511F8014B03F8C8
:10582000014F9142F9D110BD02440346934200D189
:10583000704703F8011BF9E7034611F8012B1846DE
:1058400003F8012B002AF8D17047000030B50B4D4A
:10585000044614F8013B5A5D02F00302012A11F8D4
:10586000012BA85C00F0030008BF2033012808BF0B
:105870002032981A01D1002AEBD130BD30660008E1
:1058800010B50B4662B1013A08D013F8014B00F88D
:10589000014B002CF7D1581A013810BD00220270BC
:1058A00013F8012B002AFBD1F5E7034613F8012B6F
:1058B000002AFBD1181A01387047024600230068FD
:1058C00000F000B8F0B508B9106888B10446204669
:1058D00014F8015B0F4617F8016B1EB965B9156026
:1058E000284605E0B542F6D1002BF0D114600370D4
:1058F000F0BD1C460CE015B914F8013B0E4616F835
:10590000015BAB42F7D1002BF3D0002304F8013C3C
:105910001460EDE7012B2DE9F047804601D0242BE0
:1059200006D900F0BFF8162303600020BDE8F08719
:10593000354F0D46284615F8014BE65D16F0080672
:10594000F8D12D2C2FD12C780126851C002B57D077
:10595000102B09D1302C07D1287800F0DF0058280F
:1059600049D16C781023023506F1004E0EF1FF3E4E
:105970000027BEFBF3F9384603FB19EAA4F1300C0B
:10598000BCF1090F14D86446A34222DD002F1DDBB1
:1059900081451BD301D1A24518DB00FB0340012741
:1059A00015F8014BEAE72B2C04BF2C78851CCDE7BA
:1059B000A4F1410CBCF1190F01D8373CE4E7A4F184
:1059C000610CBCF1190F04D8573CDDE74FF0FF37ED
:1059D000E6E7002F07DA2223C8F800307046002AD5
:1059E000A4D0691E05E006B14042002A9ED0002FD7
:1059F000F7D111609AE73024002BB5D10823B3E723
:105A0000302CA9D00A23AFE73066000813460A46B7
:105A1000014602480068FFF77DBF00BF9C010020DF
:105A2000F0B51F4C8BB005460B466E4604F1200CBA
:105A300020686168374603C7083464453E46F7D19D
:105A400021793971911E2068386022294FF00001B8
:105A500004D919700B4618460BB0F0BD581E844689
:105A6000B5FBF2F70DF1280E02FB175676440C46F3
:105A700016F8286C0CF8016F2E46B24201F10101B4
:105A80003D46EDD900225A541919A51AAA42E2DA64
:105A900010F8015F0E780670013201F80159F4E741
:105AA0000A660008014B1868704700BF9C0100207F
:105AB000FEE7704710B5164B164A17498B4218D3AC
:105AC0000021164A934217D38023154A9B00116880
:105AD000144C0B431360144B9C420FD3134C144BC8
:105AE0009C420ED3FEF784FC124C134B9C420BD30A
:105AF00010BD01CA01C3E1E702C3E3E708CC984740
:105B0000E9E708CC9847EAE708CC9847EDE7C046B4
:105B10004801002030670008000200204C070020E8
:105B200014ED00E0306700083067000830670008B7
:105B3000306700083067000830670008014B024AF0
:105B40001A60FEE70CED00E00400FA05044A430980
:105B50009B009B181F2210401E3A82401A6070471B
:105B600000E100E010B51F2812D90F2318400438B7
:105B7000C0B28308084A9B001824C0002040E734C4
:105B8000844081409B181A68A2431143196010BDDC
:105B90008308024A9B00EFE718ED00E000E400E014
:105BA000514161005B01610167016D017301790180
:105BB0007F0185018B01910197019D01A301A8013E
:105BC000AE01B401BA01C001C601CB01D101D701B8
:105BD000DC01E201E701ED01F201F801FD01020241
:105BE00008020D02120217021C02210226022B02D9
:105BF0003002350239023E02420247024B02500295
:105C0000540258025C026002640268026C026F0275
:105C1000730276027A027D028002840287028A027F
:105C20008C028F0292029502970299029C029E02B8
:105C3000A002A202A402A602A802A902AB02AC0220
:105C4000AD02AF02B002B102B202B202B302B402BC
:105C5000B402B502B502B502B502B502B502B5028D
:105C6000B402B402B302B202B202B102B002AF0295
:105C7000AD02AC02AB02A902A802A602A402A202D3
:105C8000A0029E029C0299029702950292028F0244
:105C90008C028A028702840280027D027A027602E6
:105CA00073026F026C026802640260025C025802B6
:105CB000540250024B02470242023E0239023502B0
:105CC00030022B02260221021C02170212020D02D0
:105CD00008020202FD01F801F201ED01E701E20113
:105CE000DC01D701D101CB01C601C001BA01B40169
:105CF000AE01A801A3019D01970191018B018501CE
:105D00007F01790173016D01670161015B0154013C
:105D10004E01480142013C01360130012A012401B3
:105D20001E01180112010D0107010101FB00F50020
:105D3000EF00EA00E400DE00D900D300CE00C80086
:105D4000C300BD00B800B300AD00A800A3009E00D2
:105D5000990094008F008A00850080007C00770005
:105D600073006E006A00650061005D005900550017
:105D700051004D004900460042003F003B00380002
:105D8000350031002E002B002900260023002000C2
:105D90001E001C00190017001500130011000F0051
:105DA0000D000C000A0009000800060005000400B0
:105DB00003000300020001000100000000000000D9
:105DC00000000000000000000100010002000300CC
:105DD0000300040005000600080009000A000C008A
:105DE0000D000F00110013001500170019001C0012
:105DF0001E0020002300260029002B002E00310069
:105E0000350038003B003F004200460049004D008D
:105E10005100550059005D00610065006A006E0088
:105E2000730077007C00800085008A008F0094005A
:105E300099009E00A300A800AD00B300B800BD000B
:105E4000C300C800CE00D300D900DE00E400EA00A1
:105E5000EF00F500FB00010107010D01120118011F
:105E60001E0124012A01300136013C014201480192
:105E70004E0154012E00300020090D0A00557361B7
:105E800067653A0A696E666F0A73686F770A6765B5
:105E900074203C706172616D3E0A736574203C70C1
:105EA0006172616D3E203C76616C75653E0A73617E
:105EB00076650A72657365740A706C6179203C6D51
:105EC000757369633E205B3C766F6C756D653E5DF6
:105ED0000A7468726F74203C76616C75653E0A6264
:105EE0006565700A00455343617065333220726501
:105EF0007600205B005D0A54656D703A2000432CEB
:105F0000206578742000430A566F6C743A2000565E
:105F10000A437572723A2000410A4373756D3A2044
:105F2000006D41680A4552504D3A200061726D0083
:105F300064616D7000726576646972006272757377
:105F40006865640074696D696E670073696E655F8A
:105F500072616E67650073696E655F706F776572F9
:105F600000667265715F6D696E00667265715F6D66
:105F7000617800647574795F6D696E006475747919
:105F80005F6D617800647574795F7370757000641B
:105F90007574795F72616D7000647574795F726198
:105FA000746500647574795F647261670064757408
:105FB000795F6C6F636B007468726F745F6D6F6490
:105FC00065007468726F745F726576007468726FD2
:105FD000745F62726B007468726F745F73657400D3
:105FE0007468726F745F63616C007468726F745F61
:105FF0006D696E007468726F745F6D6964007468B7
:10600000726F745F6D617800616E616C6F675F6D58
:10601000696E00616E616C6F675F6D617800696EBB
:106020007075745F6D6F646500696E7075745F6321
:106030006869640074656C656D5F6D6F646500749C
:10604000656C656D5F706869640074656C656D5F33
:10605000706F6C65730070726F745F7374616C6CD9
:106060000070726F745F74656D700070726F745F32
:1060700073656E730070726F745F766F6C7400700E
:10608000726F745F63656C6C730070726F745F63C2
:10609000757272006D7573696300766F6C756D65EE
:1060A00000626561636F6E00626563006C65640029
:1060B0004F4B0A004552524F520A0068656C7000FF
:1060C000696E666F0073686F77006765740073614F
:1060D000766500726573657400706C617900746830
:1060E000726F74006265657000000000BB6000089C
:1060F000C0600008C5600008CA600008DC5F0008D6
:10610000CE600008D3600008D9600008DE60000897
:10611000E4600008000000002C5F0008305F000809
:10612000355F00083C5F0008445F00084B5F0008D3
:10613000565F0008615F00086A5F0008735F00082F
:106140007C5F0008855F00088F5F0008995F00088A
:10615000A35F0008AD5F0008B75F0008C25F0008DA
:10616000CC5F0008D65F0008E05F0008EA5F000827
:10617000F45F0008FE5F0008086000081360000874
:106180001E60000829600008346000083F600008B5
:106190004A60000856600008616000086B600008F3
:1061A000756000087F6000088A600008946000083D
:1061B0009A600008A1600008A8600008AC600008B0
:1061C00000000000191B12131D1516171A090A0BDF
:1061D0001E0D0E0F474300633600462332453244FE
:1061E00032433200472341234723412347233200D0
:1061F0004723412347234123462332472332004785
:10620000234123472341234532462332472332008B
:106210004723412347234123443245324623324713
:10622000233200472341234723412343324432454D
:106230003246233247233200454700464100474259
:1062400000414223006144474500000038620008D5
:106250003B6200083E620008416200084562000897
:10626000EA320E024C554D454E4945523100000070
:106270000000000001010000100008183001640F48
:10628000001E0000000064000100E803DC05D007E8
:106290006400800C000000000E0000000000000000
:1062A00000006466612300000000000000000000A0
:1062B00000000000000000000000000000000000DE
:1062C00000000000000000000000000000000000CE
:1062D00000000000000000000000000000000000BE
:1062E00000000000000000000000000000000000AE
:1062F000000000000000000000000000000000009E
:10630000000000000000000000000000000000008D
:10631000000000000000000000000000000000007D
:10632000000000000000000000000000000000006D
:10633000000000000000000000000000000000005D
:10634000000000000000000000000000000000004D
:10635000000000000000000000000000000000003D
:10636000000000000000000000000000000000002D
:10637000000000000000000000000000000000001D
:10638000000000000000000000000000000000000D
:1063900000000000000000000000000000000000FD
:1063A00000001932000035192B321E2CD76100086D
:1063B000E1610008DF610008DD610008DA610008C2
:1063C000E4610008F0610008FF6100081062000845
:1063D000236200080000000001020102030205021E
:1063E00006020202700B000410020002300B0005CE
:1063F000B73B5D3833353832652FBC2C3A2ADB2762
:106400009E2582238321A11FDB1D00D57FAAFE2BA1
:10641000815429FC5683D702A87D52872DF8AC7988
:10642000D3067BAE04D18550FA2FA471DB0E5A8FB0
:1064300025F08D58F22773A60CD9F623895C08DD68
:1064400077A2DF0AA07521F45E8B9D48E23763B620
:106450001CC9B461CB1E4A9F35E0CF1AB06531E448
:106460004E9BE633994C18CD67B239EC4693C71270
:10647000B86D10C56FBAEE3B91446BBE14C1954028
:10648000EA3F42973DE8BC69C316EF3A904511C414
:106490006EBBC613B96C38ED4792BD68C217439600
:1064A0003CE99441EB3E6ABF15C04B9E34E1B560B8
:1064B000CA1F62B71DC89C49E33619CC66B3E732E0
:1064C000984D30E54F9ACE1BB16472A70DD88C5908
:1064D000F3265B8E24F1A570DA0F20F55F8ADE0BC0
:1064E000A17409DC76A3F722885DD603A97C28FD78
:1064F0005782FF2A805501D47EAB8451FB2E7AAFA0
:1065000005D0AD78D20753862CF900070E091C1B65
:106510001215383F363124232A2D70777E796C6B23
:106520006265484F464154535A5DE0E7EEE9FCFB93
:10653000F2F5D8DFD6D1C4C3CACD90979E998C8B83
:106540008285A8AFA6A1B4B3BABDC7C0C9CEDBDCF3
:10655000D5D2FFF8F1F6E3E4EDEAB7B0B9BEABACE3
:10656000A5A28F88818693949D9A2720292E3B3C53
:1065700035321F18111603040D0A5750595E4B4C43
:1065800045426F68616673747D7A898E87809592C3
:106590009B9CB1B6BFB8ADAAA3A4F9FEF7F0E5E2A3
:1065A000EBECC1C6CFC8DDDAD3D4696E6760757213
:1065B0007B7C51565F584D4A4344191E1710050203
:1065C0000B0C21262F283D3A33344E494047525573
:1065D0005C5B7671787F6A6D64633E393037222563
:1065E0002C2B0601080F1A1D1413AEA9A0A7B2B5D3
:1065F000BCBB9691989F8A8D8483DED9D0D7C2C5C3
:10660000CCCBE6E1E8EFFAFDF4F330313233343548
:10661000363738396162636465666768696A6B6CCE
:106620006D6E6F707172737475767778797A000019
:106630002020202020202020202828282828202032
:10664000202020202020202020202020202020204A
:1066500088101010101010101010101010101010C2
:1066600004040404040404040404101010101010A2
:10667000104141414141410101010101010101017B
:1066800001010101010101010101011010101010AF
:10669000104242424242420202020202020202024C
:1066A0000202020202020202020202101010102074
:1066B00000000000000000000000000000000000DA
:1066C00000000000000000000000000000000000CA
:1066D00000000000000000000000000000000000BA
:1066E00000000000000000000000000000000000AA
:1066F000000000000000000000000000000000009A
:106700000000000000000000000000000000000089
:106710000000000000000000000000000000000079
:106720000000000000000000000000000000000069
:10673000FFFFFFFFFFFFFFFF0000FFFF0000FFFF65
:10674000FFFF0000FFFF0000FFFFFFFF0000FFFF53
:106750000000FFFF0000FFFFFFFFFFFF0000000041
:1067600000000000FFFFFFFFFFFFFFFFFFFFFFFF35
:10677000FFFFFFFFFFFFFFFFFFFFFFFFFFFFFFFF29
:10678000E40C0000A0010020000000000000000058
:1067900000000000000000000000000000000000F9
:1067A00000000000000000000000000000000000E9
:1067B00000000000000000000000000000000000D9
:1067C00000000000000000000000000000000000C9
:1067D00000000000000000000000000000000000B9
:0867E0000000000000000000B1
:0400000508005AB5E0
:00000001FF
